:1000000065EF06F0CFEF01F004EF08F049EC06F0E1
:10001000FF0000F000F012000CEF08F018EF00F005
:10003000F26AFC6A02EC06F004006FEC01F04AEC94
:1000400005F083EC05F026EC00F0F6D7060E41181B
:10005000D8B465B21200375001E01CD10D010CBFBD
:100060001200400E476E600E5EEC04F0010E376E1B
:10007000276A286A2750A10FD96EDA6A000EDF6E50
:10008000274A282A285005E1400E275CD8B01200E4
:10009000F1D71200020EA16F3A0EA26F010EA36FEC
:1000A000A46FA56B100EA66FA76BA86B000E112492
:1000B000A96FF00E1220AA6FFF0E1320AB6FFF0E78
:1000C0001420AC6F030EAD6FF80EAE6FAF69010E6A
:1000D000B06FB16B080EB26FB36BB46BB56BB66932
:1000E000A50EDA6F0D0110BFA50CF5D88EEC04F04B
:1000F000376A1200615106E17F0E3B6EF80E116EF9
:10010000126802D0BAEC05F0C5EC05F0F1D7286A08
:10011000040E276E0CD068EC06F027C048F028C00B
:1001200049F0BCEC04F06FEC01F0274A282A3B5060
:10013000526E536A522A000E53225250275C53507B
:100140002858D6E2E8D715280EE116280CE1172822
:100150000AE1182808E161C015F062C016F063C01A
:1001600017F064C018F015506119C2E116506219F9
:10017000BFE117506319BCE118506419B9E1276A4F
:10018000286A1AD06551A0082724D96EDA6AE20ECF
:100190003824E16EE26A000EE222DFCFE7FF382A60
:1001A000152A000E1622172218223A0E381802E1DC
:1001B00027EC04F0274A282A000185D899E2E2D7E3
:1001C00027EC04F0C0EC05F093D7070EA16F61C0D7
:1001D000A2F062C0A3F063C0A4F064C0A5F065C043
:1001E000A6F063C0F8FF62C0F7FF61C0F6FF276AA0
:1001F000286A0BD0090000016551E1082724D96E57
:10020000DA6AF5CFDFFF274A282A5DD8F3E30D012C
:1002100010BF120060D88EEC04F06AD729EC02F00F
:1002200067D70C0EA16F010EA36F020EA26F160E00
:10023000F66E7EEC05F0F5CFA4F00A00F5CFA5F040
:10024000060EA66F100EA76FA86BA96B600EAB6FA2
:100250000D0EAA6FAC6B040EAD6F000EAE6BAF6BE4
:10026000B069B169B269B369B469B569B669B769AA
:10027000B86BB96BBA6BBB6BBC6BBD6BBE6BBF6B4A
:100280000D0110BF120027D88EEC04F031D706EC18
:1002900000F02ED700016051020A01E1FBD6010AED
:1002A00001E128D7070A01E132D7010A01E14BD762
:1002B000030A86E0010A89E00F0AE9E0010AAEE0DC
:1002C000050AAFE015D76551526E536A5250275C4C
:1002D000535028581200400E476EA10E120058ECE1
:1002E00006F0415001E1120062B42DEC06F065B257
:1002F000120062B029EC05F062B8F2EC05F0030ED2
:10030000416001D0030C3C6A62A61200645064CFC5
:100310004AF07C0E4A162AE164B202D02B6A02D05F
:10032000040E2B6E0D0E2C6E62962BC0D9FF2CC0C6
:10033000DAFFDF30E8320F0B0D0A20E1336A23D8F1
:10034000DECF4AF0DDCF4BF04AC0D9FF4BC0DAFF19
:100350003350010F1FD817D8DE2A000EDD22332AB2
:10036000070E3364ECD79DEC05F008D0040E64183A
:1003700004E1629608EC05F001D062963C2A030E77
:100380003C64C2D7030C20EE02F02B50D9262C502F
:10039000DA221200E16EE26ADFCFE7FF12000150BD
:1003A0001F0BE80601E01200055001E01200060EE6
:1003B000021814E01AD0020E3D6E4A0E3FD8306A81
:1003C000090E0AD0020E3D6E450402E1870E36D8B2
:1003D00045040AE1306A1D0E2F6E06D00450210A32
:1003E000EAE0030AEFE0010A42820138E832030B37
:1003F000E80614E01200020E3D6E440E206E24D07A
:10040000020E3D6E04C044F0020C020E3D6E430E1F
:10041000F5D7020E3D6E03C043F0020C0250010AF4
:10042000D8B41200030AE7E0010AEFE00A0AD8B4E0
:100430001200030AE5E0010AECE01200206E2050F1
:10044000D8A40F0E216E1200216A4292010E2F6E67
:10045000010C4F6A100E506E516A296A2A6A4FC009
:10046000F6FF50C0F7FF51C0F8FF42D80800F5CFA3
:10047000DFFF4F2A000E50225122294A2A2A040E59
:100480002A5CEDE30D0EE8CFE8F0600EE8CFE9F06E
:10049000000E496E040E486EBCEC04F04F68130E5B
:1004A000506E516A030E2A6E296851C0F8FF50C081
:1004B000F7FF4FC0F6FF1CD8DF50F56E0C0029C0C7
:1004C0004EF03F0E4E1607E168EC06F0040EA66EE5
:1004D000B50EDEEC05F04F06000E505A515A0A00D8
:1004E00029502A1001E112002906D8A02A06DDD7DA
:1004F000E20E2924D96E000E2A20DA6E12000304BF
:100500000BE101501F0B08E1010E3D6E030E0218B6
:1005100002E1428001D042900350D8A41200015061
:100520001F0B020AD8A4120005500F0BD8B41200FA
:1005300033D8476A0D0E486E040E4726000E482237
:10054000F3504726F450482221D847241D6EF4501A
:1005500048201E6E030E021807E113D8040EDF6E4A
:1005600010D8000EDB8E000C05AE04D00AD8400E69
:10057000DF6E400C06D8080EDF6E03D8000EDB8E4F
:10058000000C1DC0D9FF1EC0DAFF1200010E05AE1F
:10059000000E040DF3501200010E3D6E05500F0BBE
:1005A000080D12003D5010E124EC05F0196E3A04DC
:1005B00005E1010EE4EC04F03A6A1200000EE4ECEE
:1005C00004F0010E3A6E010C01AE1ED0010E3E6E1B
:1005D0002F50075C3050085804E207C02FF008C0C5
:1005E00030F023EC03F0480E196E010EE4EC04F039
:1005F000000EE4EC04F0240E0D010A6F0D0E0B6FDB
:10060000480E086F088F480C020E3E6E040E196EDD
:100610000750081002E1480E196E3A0405E1010E78
:10062000E4EC04F03A6A05D0000EE4EC04F0010EAC
:100630003A6E07500810D8A412000D01096B480E3D
:10064000086F088F480C080E326E30500DE1080E0E
:100650002F5C0AE22FC032F0405002E1010E03D0BD
:10066000400402E1020E406E32C009FD32502F5E9E
:10067000000E305A240E1D6E0D0E1E6E42A21AD0B0
:100680000BD01BD8C1EC02F00E0EF76403D00800AB
:10069000F55001D019D81ED83250F3E112000DD810
:1006A000C1EC02F00E0EF76403D00800F55001D043
:1006B0000BD810D83250F3E1120020C0F6FF21C051
:1006C000F7FF000EF86E1200F6CFE1FFF7CFE2FF62
:1006D000E7501200DF6E1D4A1E2A204A212A3206E8
:1006E00012000138E832030B18E01200010E3D6ED3
:1006F000040E416E040C010E3D6E450E206E24EF7B
:1007000002F02CD8496E49C020F024EF02F026D820
:10071000D96EDA6A03C0DFFF1200025002E1EFEF88
:1007200003F0010A02E17FEF02F0020A02E17FEF2B
:1007300002F0060ADBE0030A02E1B3EF03F0010A6C
:10074000D8B412000F0AD7E0010A02E1DEEF07F089
:10075000030AD7E0010ADBE0070A1200010E3D6E32
:100760000550460F1200800E011830E01200010EF5
:100770003D6EA40E1EEC02F0120E09D003502DE1C6
:10078000010E3D6E380E1EEC02F0306A290E2F6EFF
:1007900024D0010E3D6E0350010F476E47C0F6FF97
:1007A0000F0EF76E000EF86E0900F5CF20F00F0E59
:1007B000216E5DEC03F00E0EF76403D00800F550D7
:1007C00002D064EC03F02F6E306A07D00450010AA7
:1007D000CEE0030AD3E0010ADCE042821200246B7F
:1007E000256B23D0010E3D6E42B0248325D0010E2F
:1007F0003D6E22D0CCEC02F0476A0D0E486E040E1E
:100800004726000E4822F3504726F4504822C6ECF3
:1008100002F047241D6EF45048201E6EC1EC02F019
:10082000DFA40AD0010E246F07D001501F0BDAE0BD
:10083000010ADDE0030ADEE03D04D8A41200240E24
:10084000206E0D0E216E4292020E2F6E020C366A41
:1008500027D03850486E000E48BEFF0E496E4A6ED3
:100860004B6E4850155C0D6E495016580E6E4A502E
:1008700017580F6E4B501858106E0FC0F8FF0EC06F
:10088000F7FF0DC0F6FF11D80D00362A0ED80C0068
:10089000362A240EA66EB50EDEEC05F0FE0E3826C6
:1008A0003850800A7F0FD5E21200E20E3624D96E4E
:1008B000DA6A000EDA22DF50F56E1200496E3F6AE6
:1008C0000D010CBF120047500D5D02E20DCD47F047
:1008D0003F6A0BD02C0E3F24D96EDA6A0D0EDA2255
:1008E00049503F24CAEC01F03F2A47503F5CF2E3F5
:1008F000400E0D010D6F0C170CBD03D0486A482A3D
:1009000001D0486A483A484648460D010C514818FB
:10091000BF0B48180C6F0C870C8F1200496E400EED
:10092000476401D0476E4A6A0DD049504A24D96EB7
:10093000DA6A6C0E4A24E16EE26A0D0EE222DFCF23
:10094000E7FF4A2A47504A5CF0E347C011FD400EDA
:100950000D01101710BD03D0486A482A01D0486A1B
:10096000483A484648460D0110514818BF0B4818F0
:10097000106F1087108F1200495006E1040E485C7A
:1009800003E2496A040E486E48504A6E49504B6E65
:100990004C6A4D6A0A0ED8904A364B364C364D3664
:1009A000E82EF9D74AC009F04BC00AF04CC00BF052
:1009B0004DC00CF00BC0F8FF0AC0F7FFF66A140E2A
:1009C000A66EB50EDEEF05F0476E080E1A6E1C0E11
:1009D0001B6E0D0E1C6E475006E1140E1B6E0D0EA5
:1009E0001C6E256A03D0040E256E0D0E266E0BD8E4
:1009F00019C0DEFF1AC0DEFF1BC0DEFF1CC0DEFF19
:100A000002D8DF8E120025C0D9FF26C0DAFF1200FF
:100A1000040E411808E103C038FF0F013851050EDC
:100A2000D8B4030E416E3E04D8A4120023EC03F0A8
:100A3000020E401802E108D8040C0D01480E08BD52
:100A4000080E086F088F1200040E0D01086F088F42
:100A5000040C030E416E0F01376B626A7B0E366F1A
:100A6000386BF8EC07F0160E266F658C03D0629693
:100A700068EC06F062B6FBD7659C6598040E196EAB
:100A8000000EE4EC04F0010E3A6E426A456A000E74
:100A900041EF06F02306D8A0240623502410D8A442
:100AA00012004E0E246E236A060E416002D08B8423
:100AB000060C8BB403D0476A472A01D0476A4746E1
:100AC00047468B504718FB0B47188B6E1200060EDB
:100AD000F66E14D80D0EF5180DE10900600EF5182C
:100AE00009E1F66A0BD8F52803E10900F52802E0D0
:100AF00000EF08F018EC00F000EF00F0100EF76EB9
:100B0000F86A0900100CC0BC1200030ED36E659287
:100B10006596F26A0ED808D0C0AC04D02D06D8A0D5
:100B20002E0601D006D804002D502E10F5E1FF004E
:100B30001200040E2E6E2D6A040C0D01086B406A23
:100B400000AF02D0006B3A6A04AF03D0046B010E11
:100B50003A6E3E6A3D6A2F6A306A659871EC03F01E
:100B600002EC00F0D2EF02F005D80FD8376A08D8AF
:100B7000386A12007E0E3B6E116AFC0E126EFC0C7F
:100B800015681668176818681200010E136E146A4B
:100B9000000C3F6A1E0E0F01276F400E0D010D6FF6
:100BA0002C0E0E6F0D0E0F6F080E0C6F0C8F6C0E4F
:100BB000126F0D0E136F400E106F400C476EF29EB9
:100BC00083EC05F0B50E471804E0030ED36E030066
:100BD000FED7550EA76EAA0EA76EA682A6B2FED7A6
:100BE000A694120036CF35F0040E0F01366F6298CE
:100BF0006582A198A08822EC06F0A09835500F01DC
:100C000036131200600ED36E9B8C54EC06F037EC5A
:100C100006F00F01486B496BB4EC05F08B9494948B
:100C20005FEF06F0390402E149EC06F0656A150E43
:100C30000F01396F366B658629EC05F0010E416EA8
:100C4000396A12008B94D3CF31F00300A1B802D0DF
:100C5000D0A6FBD731C0D3FF120051EC06F065924D
:100C60000F01369501D0629462A41200FCD705D022
:100C700068EC06F04706D8A0480647504810F8E14F
:100C80001200476E4704D8A41200C9EC05F0B4EF77
:100C900005F06592656A4868476837EC06F0416A76
:100CA000120002D83DEF06F0030E486E476A030CAF
:100CB000390401E1120065A612EC06F0120065B6D7
:100CC00049EC06F0396A58EF06F0000167EF05F0CD
:080CD0000400120012001200E2
:100F000000B6046134034D006900630072006F0095
:100F100063006800690070002000540065006300F1
:100F200068006E006F006C006F00670079002000A1
:100F300049006E0063002E000902290001010080B3
:100F40003209040000020300000009211101000120
:100F5000221D000705810340000107050103400031
:100F60000126034800490044002000550053004278
:100F700000200042006F006F0074006C006F006181
:100F8000006400650072000600FF0901A10119015B
:100F90002940150026FF0075089540810019012998
:100FA000409100C01201000200000008D8043C007B
:100FB000010101020001040309040000010E3D6E5D
:100FC0000F0116D8346A3450460FD96EDA6ADF6AD8
:100FD000342A3450F8E003C045F0455041EC06F0A7
:100FE000035003E1050E416E050C060E416E060C22
:100FF000276B286B296B2A6B2B6B2C6B2D6B1200CC
:021006000D607B
:020000040001F9
:08FFF8008CF70AFAF2F8FFFB96
:00000001FF
